:020000040000FA
:0200000067296E
:08000800F000030E8301F1007A
:100010000A08F2008A01F3080319562883128601A0
:1000200087018801890183160130860088018901D2
:10003000C030870083122E08FE39860089012E18F1
:10004000091530083F398700301B0914B01B89148B
:100050002C088800051000000000F30300000000D9
:100060000514031949282F08FE39860089012F1825
:10007000091531083F398700311B0914B11B891458
:100080002D088800051000000000F30100000000AA
:100090000514831286018701880189018316FF30C8
:1000A00086008700880007308900831272088A0062
:1000B000710E8300F00E700E8B100B160900831268
:1000C0008601870188018901831601308600880135
:1000D000C0308700890183120800831286018701DE
:1000E000880189018316FF30860087008800073069
:1000F0008900831286018701880189010800F308BD
:10010000031987287308013C03198F287F282708C3
:10011000AC002508B0002308AE00F30A0800270849
:10012000AD002508B1002308AF00F30A0800A301C1
:10013000A501AB01A7017F20A30AAB0AAB1E9A2839
:10014000AB012430A7007F20A30AAB0AAB1EA12875
:10015000AB014930A7007F20A30AAB0AAB1EA92838
:10016000AB016E30A7007F20A30AAB0AAB1EB128FB
:10017000AB019230A7007F20A30AAB0AAB1EB928BF
:10018000AB01B730A7007F20A30AAB0AAB1EC12882
:10019000AB01DB30A7007F20A30AAB0AAB1EC92846
:1001A000AB01FF30A7007F20A30AAB0AAB1ED1280A
:1001B000AB01A301A50AA51F9A28FF30A7007F2045
:1001C000A30AAB0AAB1EDD28AB01DB30A7007F2002
:1001D000A30AAB0AAB1EE528AB01B730A7007F200E
:1001E000A30AAB0AAB1EED28AB019230A7007F201B
:1001F000A30AAB0AAB1EF528AB016E30A7007F2027
:10020000A30AAB0AAB1EFD28AB014930A7007F2033
:10021000A30AAB0AAB1E0529AB012430A7007F203F
:10022000A30AAB0AAB1E0D29AB01A7017F20A30ACD
:10023000AB0AAB1E1529AB01A50FDD28A301A50153
:10024000080023084F3C031C2C298313A0302307EC
:10025000840026088000080023089F3C031C3829DE
:100260008317D030230784002608800083130800FA
:100270002308FF3C031C08008317F0302307840089
:10028000260880008313080023084F3C031C4F29D5
:100290008313A030230784000008A6000800230869
:1002A0009F3C031C5B298317D03023078400000880
:1002B000A600831308002308FF3C031C08008317D3
:1002C000F030230784000008A6008313080083127F
:1002D000031385019F01831606309F008501831259
:1002E000013085006D20981783160C309900181581
:1002F00018128312A201F301A301A401A5018B1717
:100300000B178316011783120B16181385159720E8
:100310001816A301A401A801A901F308031D8D2942
:1003200085118C1E912985151A08A200A2080319AF
:10033000C829A808031DA803A908031DA903A40828
:10034000031DAA29A5012208A60021212208A70031
:100350007F20C029A001A00CA0012408A500A50DA4
:100360002208A7007F20442126082207A100A10C13
:10037000A5032108A7007F207F202208A6002121B5
:100380002308FF3C03198D29A30F8D29A3038D2971
:10039000A80AA90A28080A3C0318D7292308E63C1A
:1003A0000318D729A801A301A40AA41BA4032908A0
:1003B000643C03188D29A401A301A901A8018D297A
:02400E00B23FBF
:00000001FF
